:020000040000FA
:04000000E8303A2882
:040004000034003490
:08000800A000030EA100831209
:1000100005191128831601178312B2308100B1012E
:100020002C2883160113831203140B190310A80D37
:10003000A90DAA0DAB0DAC0DAC16FF302C02031DA3
:100040002C28FA302B02031D2C2832152A08AF0069
:100050002908AE002808AD008B100B11210E83007B
:06006000A00E200E0900B5
:0C007400203084008001840A80300402E7
:10008000031C3C28EF2183160C3085058701831261
:10009000850187010730990000309A0010308316DF
:1000A0008E008312603083168F0083120030831617
:1000B000910000008312C830831681008312313012
:1000C0009000003083168C00831210308B00462382
:1000D00081018E018F010B118B100B108C018B177E
:1000E0007F2032198B20B40B7D280310851903144F
:1000F000BA0DF0303A0203194621E3237028640058
:100100003310B10A311F8A28AC01AB01AA01A90141
:10011000A801B101080032110130B7008B13203063
:10012000370783169B001C141A088312A400103092
:10013000370783169B001C141A088312A300A6001D
:100140000230A6060030370783169B001C141A08DD
:100150008312A200A7000130A7068B17331CB62814
:1001600022090339A200A309A409A50924082F0222
:10017000031D402923082E02031D402922082D02B9
:10018000031D402901303702031DCB283E18CB2820
:100190003E143F140A2202303702031DD428BE1831
:1001A000D428BE143F141D2203303702031DDD285E
:1001B0003E19DD283E153F14302204303702031D5E
:1001C000E628BE19E628BE153F1443220530370243
:1001D000031DEF283E1AEF283E163F145622063024
:1001E0003702031DF828BE1AF828BE163F146922EC
:1001F00007303702031D01293E1B01293E173F141A
:100200007C2208303702031D0A29BE1B0A29BE17AB
:100210003F14882209303702031D13295E18132961
:100220005E143F1494220A303702031D1C29DE1885
:100230001C29DE143F14A2220B303702031D25298E
:100240005E1925295E153F14B0220C303702031DBC
:100250002E29DE192E29DE153F14BE220D3037025D
:10026000031D37295E1A37295E163F14CC220E3043
:100270003702031D4029DE1A4029DE163F14D92219
:10028000B70A0F303702031808008E280130B60075
:10029000B400B500B70085018701B21343237F2066
:1002A000B40B5F29031085190314BA0DF0303A021C
:1002B00003198729B50B5F299630B5009321321DAC
:1002C0004F293211331C69292D090339AD00AE09BC
:1002D000AF092F1C4F292D08300203194F292D0873
:1002E000B0002E1E4F298B1320303707BC002F087B
:1002F000BB00DA2110303707BC002E08BB00DA2122
:1003000000303707BC002D08BB00DA218B178501B0
:100310008701B70AB6010130B5000F303702031C60
:100320004F2946230800013037020319FD2202300D
:10033000370203190223033037020319072304305D
:10034000370203190C230530370203191123063035
:100350003702031916230730370203191B2308300D
:1003600037020319202309303702031925230A30E5
:10037000370203192A230B30370203192F230C30BD
:100380003702031934230D303702031939230E3095
:10039000370203193E2308003F1C08003F101030AD
:1003A000BC003E08BB00DA213030BC005E08BB0058
:1003B000DA2108008B133B0883161C159A00831260
:1003C0003C0883169B0055309D00AA309D009C146C
:1003D00064009C18E8291C1183128B1708008316EF
:1003E00010309B001C141A088312BE008316303094
:1003F0009B001C141A088312DE00FF30C800CA15C7
:10040000CB15CC15CD15CE15CF15D015D115D215D0
:10041000D3150800C130BE05FF30DE055F1E172A68
:100420001C30C405C0000030C200C6005F101C3084
:10043000D4000030D500902B0800C230BE05FF303C
:10044000DE055F1E2A2A3330C405C0000030C2001A
:10045000C6005F103330D4000030D500902B080068
:10046000C430BE05FF30DE055F1E3D2A3930C405AD
:10047000C0000030C200C6005F103930D400003028
:10048000D500902B0800C830BE05FF30DE05DF1E0A
:10049000502A4C30C405C0000030C200C6005F10B6
:1004A0004C30D6000030D7009B2B0800D030BE0562
:1004B000FF30DE05DF1E632AC330C405C0000030F4
:1004C000C200C6005F10C330D6000030D7009B2B9F
:1004D0000800E030BE05FF30DE05DF1E762AC93099
:1004E000C405C0000030C200C6005F10C930D6008D
:1004F0000030D7009B2B08007F30BE050030DE05A2
:100500004030C505C1000030C300C700E62A08001E
:10051000BF30BE050030DE058030C505C1000030AB
:10052000C300C700F12A08003F30BE050130DE05D8
:100530009F2A0030C505C1000030C300C7005F1509
:10054000DF1508003F30BE050230DE05AD2A003061
:10055000C505C1000030C300C7005F15DF150800E6
:100560003F30BE050430DE05BB2A0030C505C100A2
:100570000030C300C7005F15DF1508003F30BE051F
:100580000830DE05C92A0030C505C1000030C300AF
:10059000C7005F15DF1508003F30BE051030DE05CF
:1005A000D72A0030C505C1000030C300C7005F1165
:1005B00008003F30BE052030DE05E42A0030C505C6
:1005C000C1000030C300C7005F1108005F1A0800B7
:1005D0005F16DF125408C405C0005508C200C600EB
:1005E0000800DF1A0800DF165F125608C405C000B5
:1005F0005708C200C6000800080003308506123004
:10060000870608003030850616308706080012304D
:1006100085061630870608000330850609308706F0
:10062000080030308506293087060800123085061C
:100630002930870608000030850616308706080036
:1006400000308506293087060800223085060030F4
:100650008706080021308506003087060800223012
:1006600085060030870608002130850600308706A1
:1006700008003230850600308706080031308506D4
:100680000030870608003E18FD220800A6235F12EE
:10069000DF12BE1BDF16DF1E5F163E180A22BE18D1
:1006A0001D223E193022BE1943223E1A5622BE1A7E
:1006B00069223E1B7C22BE1B88225E189422DE1813
:1006C000A2225E19B022DE19BE225E1ACC22DE1AE8
:1006D000D9220800B601B401B5013D1C722BBD0141
:1006E000BD14742BBD013D143D08B6006400782B89
:1006F000792B7A2B7B2B7C2BFF30B51B8500B51F0C
:100700008501B40B762BB50B762B0310B60CB6080F
:10071000031D762B0030BC003D08BB00DA21080029
:100720004030BC005408BB00DA215030BC005508F2
:10073000BB00DA2108006030BC005608BB00DA219B
:100740007030BC005708BB00DA2108008316403027
:100750009B001C141A088312D400831650309B008F
:100760001C141A088312D500831660309B001C14D9
:100770001A088312D600831670309B001C141A08C6
:100780008312D700080005125C180516DC1C8512C0
:10079000DC1885165C1D05105C190514DC1D851020
:1007A000DC1985145C1E87105C1A8714DC1E071187
:1007B000DC1A07155C1F07105C1B0714DC1F87126F
:1007C000DC1B871608008F08031908008F0178309A
:1007D0008E00C80F252EC80ADF19152C441C152CB5
:1007E000461C062CCA1CF72BCA014A15232C4A1D8D
:1007F000FC2BCA01CA15232CCA1D012CCA014A169A
:10080000232C4A1E232CCA01CA14232C4A1D0B2C4C
:10081000CA014A16232CCA1D102CCA014A16232CC1
:100820004A1E232CCA01CA14232CCA1C1A2CCA0122
:100830004A15232C4A1D1F2CCA01CA15232C4A1EF7
:10084000232CCA014A15DF194C2CC41C4C2CC61C85
:100850003D2CCB1C2E2CCB014B155A2C4B1D332C75
:10086000CB01CB155A2CCB1D382CCB014B165A2C57
:100870004B1E5A2CCB01CB145A2C4B1D422CCB01B6
:100880004B165A2CCB1D472CCB014B165A2C4B1E0A
:100890005A2CCB01CB145A2CCB1C512CCB014B1511
:1008A0005A2C4B1D562CCB01CB155A2C4B1E5A2CB7
:1008B000CB014B15DF19832C441D832C461D742C52
:1008C000CC1C652CCC014C15912C4C1D6A2CCC01F8
:1008D000CC15912CCC1D6F2CCC014C16912C4C1EA0
:1008E000912CCC01CC14912C4C1D792CCC014C16A4
:1008F000912CCC1D7E2CCC014C16912C4C1E912C95
:10090000CC01CC14912CCC1C882CCC014C15912CF6
:100910004C1D8D2CCC01CC15912C4C1E912CCC0156
:100920004C15DF19BB2CC41DBB2CC61DAC2CCD1C1B
:100930009D2CCD014D155F13C92C4D1DA22CCD0151
:10094000CD15C92CCD1DA72CCD014D16C92C4D1E82
:10095000C92CCD01CD14C92C4D1DB12CCD014D1686
:10096000C92CCD1DB62CCD014D16C92C4D1EC92C40
:10097000CD01CD14C92CCD1CC02CCD014D15C92CD9
:100980004D1DC52CCD01CD15C92C4D1EC92CCD0139
:100990004D15DF19F42C5F1BF42C441EF42C461E5D
:1009A000E52CCE1CD62CCE014E15022D4E1DDB2C77
:1009B000CE01CE15022DCE1DE02CCE014E16022DFD
:1009C0004E1E022DCE01CE14022D4E1DEA2CCE015C
:1009D0004E16022DCE1DEF2CCE014E16022D4E1EB0
:1009E000022DCE01CE14022DCE1CF92CCE014E15B7
:1009F000022D4E1DFE2CCE01CE15022D4E1E022DB7
:100A0000CE014E15DF192B2DC41E2B2DC61E1C2DFD
:100A1000CF1C0D2DCF014F15392D4F1D122DCF019C
:100A2000CF15392DCF1D172DCF014F16392D4F1E44
:100A3000392DCF01CF14392D4F1D212DCF014F1648
:100A4000392DCF1D262DCF014F16392D4F1E392D93
:100A5000CF01CF14392DCF1C302DCF014F15392D9B
:100A60004F1D352DCF01CF15392D4F1E392DCF01FB
:100A70004F15DF19622D441F622D461F532DD01CC8
:100A8000442DD0015015702D501D492DD001D01589
:100A9000702DD01D4E2DD0015016702D501E702D72
:100AA000D001D014702D501D582DD0015016702D2E
:100AB000D01D5D2DD0015016702D501E702DD0010F
:100AC000D014702DD01C672DD0015015702D501DE5
:100AD0006C2DD001D015702D501E702DD0015015E9
:100AE000DF19992DC41F992DC61F8A2DD11C7B2D6E
:100AF000D1015115A72D511D802DD101D115A72D43
:100B0000D11D852DD1015116A72D511EA72DD10123
:100B1000D114A72D511D8F2DD1015116A72DD11DF7
:100B2000942DD1015116A72D511EA72DD101D114FD
:100B3000A72DD11C9E2DD1015115A72D511DA32DDF
:100B4000D101D115A72D511EA72DD1015115DF19A6
:100B5000D12D451FD12D471FC22DD21CB32DD2013F
:100B60005215DF13DF2D521DB82DD201D215DF2D06
:100B7000D21DBD2DD2015216DF2D521EDF2DD20106
:100B8000D214DF2D521DC72DD2015216DF2DD21DDA
:100B9000CC2DD2015216DF2D521EDF2DD201D214E0
:100BA000DF2DD21CD62DD2015215DF2D521DDB2D8B
:100BB000D201D215DF2D521EDF2DD2015215DF19C1
:100BC0000A2EDF1B0A2EC51F0A2EC71FFB2DD31CA2
:100BD000EC2DD3015315182E531DF12DD301D31530
:100BE000182ED31DF62DD3015316182E531E182E72
:100BF000D301D314182E531D002ED3015316182ED3
:100C0000D31D052ED3015316182E531E182ED301B3
:100C1000D314182ED31C0F2ED3015315182E531D89
:100C2000142ED301D315182E531E182ED30153158D
:100C3000CC214008C4004108C5005F18DF145F1CC8
:100C4000DF105F19DF155F1DDF114808C9000C3088
:100C50004A05031D05120C304B05031D85120C308F
:100C60004C05031D05100C304D05031D85100C307F
:100C70004E05031D87100C304F05031D07110C3066
:100C80005005031D07100C305105031D87120C3051
:100C90005205031D07120C305305031D8711490827
:100CA0000E0203187F2E12304A05031D051612305E
:100CB0004B05031D851612304C05031D051412301B
:100CC0004D05031D851412304E05031D8714123087
:100CD0004F05031D071512305005031D0714123070
:100CE0005105031D871612305205031D07161230D9
:100CF0005305031D8715FF304802031908008F08AC
:100D0000031D08007F2049080E02031C7F2E1830A7
:100D10004A05031D051206304A05031D0516183045
:100D20004B05031D851206304B05031D8516183033
:100D30004C05031D051006304C05031D0514183025
:100D40004D05031D851006304D05031D8514183013
:100D50004E05031D871006304E05031D87141830FD
:100D60004F05031D071106304F05031D07151830E9
:100D70005005031D071006305005031D07141830D9
:100D80005105031D871206305105031D87161830C3
:100D90005205031D071206305205031D07161830B1
:100DA0005305031D871106305305031D87150800E1
:084000000D00030007000100A0
:02400E00CC33B1
:10420000010078007A007C007E007B0079007F004E
:104210007D007A0078007E007C007D007F007900C0
:104220004200F200F600FA00FE00F200F600FA008A
:10423000FE00F200F600FA00FE00F200F600FA00BE
:10424000FF00050005000500050009000900090040
:1042500009000D000D000D000D00110011001100EE
:104260000000FF00FF00FF00FF00FF00FF00FF0055
:10427000FF00FF00FF00FF00FF00FF00FF00FF0046
:1042800033007B00FF00FF00FF00FF00FF00FF0086
:10429000FF00FF00FF00FF00FF00FF00FF00FF0026
:1042A0000000FE00FF00FF00FF00FF00FF00FF0016
:1042B000FF00FF00FF00FF00FF00FF00FF00FF0006
:1042C000C3001100FF00FF00FF00FF00FF00FF0020
:1042D000FF00FF00FF00FF00FF00FF00FF00FF00E6
:1042E0000000FF00FF00FF00FF00FF00FF00FF00D5
:1042F000FF00FF00FF00FF00FF00FF00FF00DD00E8
:00000001FF
